:020000040800F2
:1000000000040020A1020008791000087D100008FB
:10001000D11000087D100008A5100008A3020008F8
:10002000A3020008A3020008A30200080529000893
:10003000A3020008A3020008A3020008A30200080C
:10004000A3020008A3020008A3020008A3020008FC
:10005000A3020008A3020008493E0008753E0008FC
:10006000A13E0008CD3E0008F93E0008A3020008AA
:10007000A3020008A3020008A3020008A3020008CC
:10008000A3020008A3020008A3020008A3020008BC
:10009000A3020008A3020008A3020008253F0008ED
:1000A000A3020008A3020008A3020008A30200089C
:1000B000A3020008A3020008A3020008A30200088C
:1000C000A3020008A3020008A3020008A30200087C
:1000D000A3020008A3020008A3020008A30200086C
:1000E0008D3F0008A3020008A3020008A302000835
:1000F000A3020008A3020008A3020008A30200084C
:10010000A3020008A3020008C53A0008A3020008E1
:10011000A3020008A3020008A3020008A30200082B
:10012000A3020008A3020008A3020008A30200081B
:10013000A3020008A3020008A3020008A30200080B
:10014000A3020008A3020008A3020008A3020008FB
:10015000A3020008A3020008A3020008A3020008EB
:10016000A3020008A3020008A3020008A3020008DB
:10017000A30200083D340008A3020008A3020008FF
:10018000A3020008A302000861110008A3020008EE
:10019000A3020008A3020008A3020008A3020008AB
:1001A000A3020008A3020008A3020008A30200089B
:1001B000A3020008A3020008A3020008A30200088B
:1001C000A3020008A3020008A3020008A30200087B
:1001D000A302000829340008A3020008A3020008B3
:1001E000A3020008A3020008A3020008A30200085B
:1001F000A3020008A3020008A3020008A30200084B
:10020000A3020008A3020008A3020008A30200083A
:10021000A3020008A3020008A3020008A30200082A
:10022000A3020008A3020008A3020008A30200081A
:10023000A3020008A3020008A3020008A30200080A
:10024000A3020008A3020008A3020008A3020008FA
:10025000A3020008A3020008A3020008A3020008EA
:10026000A3020008A3020008A3020008A3020008DA
:10027000A3020008A3020008A3020008A3020008CA
:10028000A3020008A3020008A3020008A3020008BA
:10029000A3020008A3020008A3020008A3020008AA
:1002A00002E000F000F8FEE772B6394880F30888F3
:1002B000384880F3098838484EF60851CEF20001DC
:1002C000086040F20000CCF200004EF63471CEF22D
:1002D00000010860BFF34F8FBFF36F8F40F2000043
:1002E000C0F2F0004EF68851CEF200010860BFF374
:1002F0004F8FBFF36F8F4FF00000E1EE100A4EF604
:100300003C71CEF200010860062080F31488BFF330
:100310006F8F02F035FB03F053FB4FF055301F4950
:100320001B4A91423CBF41F8040BFAE71C49194AA9
:1003300091423CBF41F8040BFAE71A491A4A1B4B99
:100340009A423EBF51F8040B42F8040BF8E7002034
:100350001749184A91423CBF41F8040BFAE702F0F2
:1003600053FB03F0A1FB144C144DAC4203DA54F8D8
:10037000041B8847F9E700F03FF8114C114DAC42DF
:1003800003DA54F8041B8847F9E702F03BBB00008E
:1003900000040020002400200000000800000020CD
:1003A00000040020F0430008002400204424002022
:1003B0004824002060350020A0020008A0020008A8
:1003C000A0020008A00200082DE9F04F2DED108AD0
:1003D000C1F80CD0D0F80CD0BDEC108ABDE8F08F7D
:1003E000002383F311882846A047002001F0E4FE93
:1003F00001F094FE00DFFEE738B5204C6FF00A03F1
:10040000002523700323A57063701A23E5702571FE
:100410006571A571E57125726572A372E57200F0D0
:1004200055FD20B10E2325726572A372E57202F0AC
:100430002BFA044602F060FA0546D0B9104B9C42F4
:1004400019D001339C4241F2883412BF0546002482
:100450000125002002F022FA0DB100F0B7F800F0FB
:10046000B1FD00F07DFC204600F070F900F0AEF820
:10047000F9E70024EDE70446EBE700BF482400203D
:10048000010007B008B500F0E9FBA0F120035842D5
:10049000584108BD054B07B51B88022101A8ADF8DE
:1004A000043000F047FC03B05DF804FB9440000802
:1004B000064991F8243033B100230822086A81F8F4
:1004C000243000F07FBC0120704700BF682400206A
:1004D0002DE9F84F234C05468846174694F82430FA
:1004E0008BBB2E46DFF87C90002F38D094F824A0E8
:1004F000BAF1000F05D12022FF214846266200F004
:100500004FFDCAF10805414604EB8A00BD4228BFF1
:100510003D465FFA85FBAD00A7EB0B072A462E444C
:1005200000F016FD94F82430A844FFB29B445FFA13
:100530008BFBBBF1080F84F824B0D5D1FFF7B8FFCF
:100540000028D1D108E0266A06EB8306B042C9D064
:10055000FFF7AEFF0028C4D10020BDE8F88F0120CE
:10056000BDE8F88F6824002010B5202383F311889C
:100570001248C3680BB101F0A5FE0023104A4FF4E6
:100580007A710E4801F062FE002383F311880D4C4E
:10059000236813B12368013B2360636813B1636868
:1005A000013B6360084B1B7833B9636823B90220B1
:1005B00000F0C4FC3223636010BD00BF542400204F
:1005C000690500089825002090240020554B5649C5
:1005D0002DE9F04153F8042F013201D1BDE8F0813B
:1005E0008B42F7D1514C524B22689A4240F298808C
:1005F000504B9B6803F1006303F500339A4280F08F
:100600008F80002000F0D6FB02204B4B187000F0CA
:100610008DFC4A4BD3F8E8200022C3F8E820D3F839
:100620001011C3F81021D3F81011D3F8EC10C3F84F
:10063000EC20D3F81411C3F81421D3F81411D3F813
:10064000F010C3F8F020D3F81811C3F81821D3F82C
:100650001811D3F8801041F00061C3F88010D3F86E
:10066000801021F00061C3F88010D3F88010D3F817
:10067000801041F00071C3F88010D3F8801021F091
:100680000071C3F88010D3F8803072B62C4B2D491E
:100690000B601D682468BFF34F8FBFF36F8F2A4B29
:1006A000C3F88420BFF34F8F5A6922F480325A6115
:1006B000BFF34F8FD3F8802043F6E07EC2F3C90624
:1006C000C2F34E32B707520102EA0E0838463146ED
:1006D000013948EA000C00F14040B1F1FF3FC3F896
:1006E00074C2F5D1203A12F1200FEDD1BFF34F8F34
:1006F000BFF36F8FBFF34F8FBFF36F8F5A6922F431
:1007000000325A610022C3F85022BFF34F8FBFF36B
:100710006F8F202383F31188AD4685F30888204727
:10072000BDE8F081FCFF01081C000208040002087B
:10073000FFFF0108482400209024002000440258B4
:100740000000020808ED00E000ED00E02DE9F04FA8
:1007500099B0B34C2022FF21019010A8A66800F0A8
:100760001FFCB04AA3461378A3B90121AE4811700B
:10077000C360202383F31188C3680BB101F0A2FD8D
:100780000023AA4A4FF47A71A74801F05FFD0023C5
:1007900083F31188019B13B1A54B019A1A600023C2
:1007A000A44AA349019F99461C461D4698461370CA
:1007B0004B600292012000F0B9FB002F00F0128282
:1007C0009B4B1B68002B40F00D8219B0BDE8F08FE9
:1007D0000220FFF757FE002840F0FB81019BB9F192
:1007E000000F08BF1F46944B1B8802210BA8ADF8D1
:1007F0002C3000F09FFADDE74FF47A7000F02EFA0B
:10080000031E0393EADB0220FFF73CFE824600282A
:10081000E4D0039B581E042800F2DD81DFE800F0DD
:10082000030E1114170018A80523042140F8343DC5
:1008300000F080FA54464FF0000856E00421784852
:10084000F6E704217D48F3E704217D48F0E71C2406
:100850002046043400F0B0FA04210B900BA800F0FD
:1008600069FA2C2CF4D1E5E7002DB7D0002CB5D0D7
:100870000220FFF707FE0546002800F0AF810120A7
:100880006C4C00F097FA4FF000090220207000F045
:100890004DFB5FFA89FA504600F09CFA074658B1C2
:1008A000504609F1010900F0A5FA0028F1D12C46C3
:1008B000A9460027634B97E701233E460220237099
:1008C00000F02AFBDBF808309E4206D2304600F0EA
:1008D00073FA0130EBD10436F4E70026029BA946F7
:1008E0002C461E703746524B5E6000F061FB15B11E
:1008F000002C18BF0027FFF7CDFD5BE7002D3FF46C
:100900006DAF002C3FF46AAF0220029B187000F01C
:100910000DFB322000F0A2F9B0F1000AC0F25E81B6
:100920001AF0030540F05A8106EB0A03DBF80820B1
:10093000934200F25381BAF5807F00F24F81554512
:100940000DDA4FF47A7000F089F90490049B002BC3
:10095000C0F24481049B3C4AAB540135EFE7C82008
:10096000FFF790FD0546002800F038811F2E11D8B2
:10097000C6F1200410AB26F0030033495445184457
:1009800028BF5446224600F0E3FA2246FF212E48B3
:1009900000F006FB4FEAAA0A2B4930465FFA8AF2BA
:1009A000FFF796FD0446002800F01A8106EB8A0640
:1009B00005469AE70220FFF765FD00283FF40EAFD9
:1009C000FFF776FD00283FF409AF4FF0000A5346C9
:1009D000DBF8082092451CD2BAF11F0F12D8109AEA
:1009E00001320FD02AF0030218A90A4452F8202C31
:1009F0000B92184604220BA90AF1040A00F07CFBB2
:100A00000346E5E75046039300F0D6F9039B0B90AD
:100A1000EFE718A8042140F84C3D00F08BF964E79B
:100A20004824002094250020542400206905000853
:100A30009825002090240020964000084C24002097
:100A400050240020984000089424002018A8002377
:100A5000642140F8343D00F039F900287FF4BEAE3F
:100A60000220FFF70FFD00283FF4B8AE0B9800F00E
:100A7000D3F918AB43F8480D04211846CDE718A860
:100A80000023642140F8343D00F020F900287FF471
:100A9000A5AE0220FFF7F6FC00283FF49FAE0B98AE
:100AA00000F0BCF918AB43F8440DE5E70220FFF76E
:100AB000E9FC00283FF492AE00F0B6F918AB43F819
:100AC000400DD9E70220FFF7DDFC00283FF486AE99
:100AD0000BA9142000F0AEF9824618A8042140F8B2
:100AE0003CAD00F027F951460BA896E7322000F004
:100AF000B5F8B0F1000AFFF671AE1AF0030F7FF4FB
:100B00006DAE0AEB0803DBF8082093423FF666AEB1
:100B10000220FFF7B7FC00283FF460AE2AF0030A7A
:100B2000C244D0453FF4E1AE404608F1040800F06D
:100B300043F904210A900AA800F0FCF8F1E74FF409
:100B40007A70FFF79FFC00283FF448AEFFF7B0FC37
:100B500000283FF4AFAE109B01330CD0082210A93F
:100B60000020FFF7B5FC00283FF4A4AE2022FF21AF
:100B700010A800F015FAFFF78DFC374801F022FBB2
:100B800023E6002D3FF42AAE002C3FF427AE18A830
:100B90000023642140F8343D00F098F88246002894
:100BA0007FF41CAE0220FFF76DFC00283FF416AE68
:100BB0000390FFF76FFC41F28830574601F002FBCB
:100BC0000B9800F039FA00F0F3F9039B1C461D4620
:100BD000F0E5054689E64FF00008FFE52546FDE50E
:100BE0002C4667E6002000F039F80490049B002BA7
:100BF000FFF6E3AD012000F08FF9049B213B122B9F
:100C00003FF6D8AD01A252F823F000BFD10700088B
:100C1000F907000869080008B5070008B5070008CB
:100C2000B5070008FD080008ED0A0008B50900082E
:100C30004D0A00087F0A0008AD0A0008B507000841
:100C4000C50A0008B50700083F0B0008EB080008BC
:100C5000B5070008830B0008A08601002DE9F347C3
:100C60004FF47A75002402AE154F4543DFF85880E3
:100C700006F8014D97F900305FFA84F95A1C01D04B
:100C8000A34212D158F82400012231460368D3F858
:100C900020A02B46D047012807D10A4B9DF807001A
:100CA00083F8009002B0BDE8F0870134022CE1D156
:100CB0004FF4FA7001F086FA4FF0FF30F2E700BF10
:100CC00000240020BC250020AC4000082DE9F0479E
:100CD0004FF47A7506460024134F4D43DFF85080D9
:100CE00097F900305FFA84F95A1C01D0A34210D161
:100CF00058F82400042231460368D3F820A02B467C
:100D0000D047042805D1094B002083F80090BDE8A6
:100D1000F0870134022CE3D14FF4FA7001F052FA5B
:100D20004FF0FF30BDE8F08700240020BC250020F4
:100D3000AC400008074B30B41A78074B53F82240F8
:100D40000A46014623682046DD69044BAC4630BCA8
:100D5000604700BFBC250020AC400008A086010011
:100D6000F8B5104C0025104E01F076FC0F4F2070A6
:100D70003068237883420CD800250D4E2078013846
:100D800001F066FC23780544013BB5422370F5D998
:100D9000F8BD01F05DFC336805440133BD423360AA
:100DA000E6D9E9E7BD250020A0250020FFFF0100CE
:100DB000FFFF030001F01CBD00F1006000F50030F2
:100DC0000068704700F10060920000F5003001F00B
:100DD0009FBC0000054B1A68054B1B789B1A834289
:100DE00002D9104401F034BC00207047A025002037
:100DF000BD25002038B5074D04462868204401F081
:100E00002DFC28B928682044BDE8384001F038BCE2
:100E100038BD00BFA025002000207047014BC058FE
:100E2000704700BF00E8F11F014B1868704700BF12
:100E30000010005C234BF0B5234C1B682788C3F3DC
:100E40000B0665681B0C94F90820BE4228D0A789C0
:100E5000BE4206D101220C2505FB0244656894F9C7
:100E6000082041F20104A3421CD041F20304A34232
:100E70001AD042F20104A34218D042F20304A34262
:100E800008BF5622441E013D0B460C44A34217D214
:100E900015F9016F581C5EB1034600F8016CF5E7C7
:100EA0000022D8E75A22EDE75922EBE75822E9E77A
:100EB0002C2584421D7001D9981C5A70401AF0BD2F
:100EC0001846FBE70010005C04240020104B41F2A0
:100ED00001015B888B429AB211D041F203018B422F
:100EE0000FD042F201039A420DD042F203039A421C
:100EF0000BD10323074A02EB8303D8787047002302
:100F0000F8E70123F6E70223F4E70020704700BF6B
:100F10000010005C9C400008022803D14FF400221E
:100F2000014B9A61704700BF00100258022802D19D
:100F30000822014B9A61704700100258022804D120
:100F4000024A536983F00803536170470010025846
:100F5000002310B5934203D0CC5CC4540133F9E7AD
:100F600010BD000030B5441E14F9010F0B4658B1F6
:100F700093F900500131854206D11AB993F9002046
:100F8000801A30BD013AEFE7002AF7D1104630BD94
:100F900002460346981A13F9011B0029FAD170473B
:100FA00002440346934202D003F8011BFAE770475C
:100FB000024B1A78024B1A70704700BFBC25002004
:100FC0000024002038B5164C164D204600F02CFCAD
:100FD0002946204600F054FC2D681348D5F890208F
:100FE000D2F8043843F00203C2F8043801F0EAF8FA
:100FF0000E49284600F054FDD5F890200C48D2F850
:1010000004380C49A04223F00203C2F804384FF41C
:10101000E1330B6003D0BDE8384000F063BB38BD5E
:10102000EC2A00208C41000840420F00B441000827
:1010300040260020A425002038B50B4B05461A7821
:101040000A4B53F822400A4B9C420CD0094B00211A
:1010500018221846FFF7A4FF056001462046BDE8A8
:10106000384000F03FBB38BDBC250020AC40000834
:10107000EC2A0020A4250020FEE7000000B59BB06C
:10108000EFF3098168226846FFF762FFEFF30583FB
:10109000034B9A6B9A6A9A6A9A6A9A6A9B6AFEE703
:1010A00000ED00E000B59BB0EFF3098168226846CF
:1010B000FFF74EFFEFF30583044B9A6B9A6A9A6A27
:1010C0009A6A9A6A9A6A9B6AFEE700BF00ED00E09E
:1010D00000B59BB0EFF3098168226846FFF738FF3F
:1010E000EFF30583034B5A6B9A6A9A6A9A6A9A6A73
:1010F0009B6AFEE700ED00E030B50A44074D9142DF
:101100000BD011F8013B09245840013CF7D040F3C3
:1011100000032B4083EA5000F7E730BD2083B8ED91
:10112000002304491A465A50C81808334260802BDD
:10113000F9D17047C0250020024A136843F0C0036C
:101140001360704700780040044B5A6810439A6857
:1011500058600AB1181D1047704700BF4026002094
:101160002DE9F84F414EF56D2F68EC6921072C628F
:1011700019D014F0080F0CBF00208020E20748BFF0
:1011800040F02000A3074FF0200348BF40F040008C
:10119000610748BF40F4807083F31188FFF7D4FFE4
:1011A000002383F31188E20509D5202383F31188F6
:1011B0004FF40070FFF7C8FF002383F311884FF04E
:1011C0002009DFF8A8A04FF0000B14F0200832D15E
:1011D0003B0615D54FF02009DFF894A020060FD567
:1011E00089F31188504600F0F1F9002830DA082020
:1011F000FFF7AAFF27F080032B60002383F31188F9
:1012000079060DD562060BD5202383F31188F26C85
:10121000336D9A4201D1336C03BB002383F31188F1
:10122000E30604D5B26E13690BB150699847BDE867
:10123000F84F01F077BB89F31188AB8C504696F8D4
:101240006410194000F05CFA8BF31188EC69BCE77C
:1012500080B2288588F31188EC69BFE727F0400742
:101260001020FFF771FF2F60D7E700BF4026002056
:101270007826002013B5104C204600F027FA04F120
:101280001400009400234FF400720C4900F0E8F8B9
:1012900004F1380000944FF40072094B094900F042
:1012A00061F9094B0C215220E365084B236602B01B
:1012B000BDE8104000F05EB840260020AC260020BB
:1012C00039110008AC2800200078004000E1F50545
:1012D000254B002908BF1946037C012B816630B5D8
:1012E00011D1224B98420ED1214BD3F8E82042F085
:1012F0008042C3F8E820D3F8102142F08042C3F8BE
:101300001021D3F810310A68036EC46D03EB520349
:10131000B3FBF2F34A68150442BF23F0070503F05C
:10132000070343EA4503E3608B6843F040036360CF
:10133000CB68510543F00103A36042F4967343F078
:10134000010323604FF0FF33236205D512F0102212
:1013500005D0B2F1805F04D080F8643030BD7F23C7
:10136000FAE73F23F8E700BFD040000840260020FE
:101370000044025800F1604300F01F0209014009D7
:1013800003F56143C9B2800083F80013012300F123
:101390006040934000F56140C0F8803103607047C1
:1013A000F8B51546826804460B46AA4200D2856805
:1013B000A1692669761AB54207D218462A46FFF770
:1013C000C7FDA3692B44A3610DE011D9AF1B3246C1
:1013D0001846FFF7BDFD3A46E1683044FFF7B8FD17
:1013E000E2683A44A261A36828465B1BA360F8BD8B
:1013F00018462A46FFF7ACFDE368E4E783689342AA
:101400002DE9F04104460F46154600D28568606913
:101410002669361AB54207D22A463946FFF798FDA3
:1014200063692B4463610EE013D9A5EB06083246CD
:101430003946FFF78DFD4246B919E068FFF788FD90
:10144000E26842446261A36828465B1BA360BDE872
:10145000F0812A463946FFF77BFDE368E2E70000AA
:1014600010B50A440024C361029B006040608460A0
:10147000C160816141610261036210BD08B582698A
:101480004369934201D1826882B9826801328260E5
:101490005A1C42611970426903699A4201D3C368B8
:1014A0004361002100F0AAFE002008BD4FF0FF308C
:1014B00008BD000070B5202304460E4683F3118852
:1014C000A568A5B1A368A269013BA360531CA361F1
:1014D00015782269934224BFE368A361E3690BB1E5
:1014E00020469847002383F31188284670BD314673
:1014F000204600F073FE0028E2DA85F3118870BD03
:101500002DE9F74F05460F4690469A46D0F81C90B5
:10151000202686F311884FF0000B144664B1224652
:1015200039462846FFF73CFF034668B9514628462E
:1015300000F054FE0028F1D0002383F31188A8EBBB
:10154000040003B0BDE8F08FB9F1000F03D00190A3
:101550002846C847019B8BF31188E41A1F4486F381
:101560001188DBE7C160816141611144C361009B67
:10157000006040608260016103627047F8B5044614
:101580000E461746202383F31188A568A5B1A368EA
:10159000013BA36063695A1C62611E702369626922
:1015A0009A4224BFE3686361E3690BB12046984720
:1015B000002080F31188F8BD3946204600F00EFE69
:1015C0000028E2DA85F31188F8BD000083694269DA
:1015D0009A4210B501D182687AB98268013282607C
:1015E0005A1C82611C7803699A4201D3C3688361E3
:1015F000002100F003FE204610BD4FF0FF3010BD6B
:101600002DE9F74F05460F4690469A46D0F81C90B4
:10161000202686F311884FF0000B144664B1224651
:1016200039462846FFF7EAFE034668B95146284680
:1016300000F0D4FD0028F1D0002383F31188A8EB3B
:10164000040003B0BDE8F08FB9F1000F03D00190A2
:101650002846C847019B8BF31188E41A1F4486F380
:101660001188DBE7026843681143016003B1184742
:10167000704700001430FFF743BF00004FF0FF3306
:101680001430FFF73DBF00003830FFF7B9BF00004E
:101690004FF0FF333830FFF7B3BF00001430FFF7CF
:1016A00009BF00004FF0FF311430FFF703BF000007
:1016B0003830FFF763BF00004FF0FF323830FFF7DC
:1016C0005DBF000000207047FFF7D4BD044B0360EE
:1016D000002343608360C36001230374704700BF2D
:1016E000E840000810B52023044683F31188FFF773
:1016F000EFFD02232374002383F3118810BD000043
:1017000038B5C36904460D461BB904210844FFF7E8
:10171000A9FF294604F11400FFF7B0FE002806DAFD
:10172000201D4FF48061BDE83840FFF79BBF38BDF6
:10173000026843681143016003B118477047000015
:1017400013B5446BD4F894341A681178042915D170
:10175000217C022912D11979012312898B4013426D
:101760000CD101A904F14C0001F09AFFD4F8944483
:101770000246019B2179206800F0EAF902B010BD11
:10178000143001F01DBF00004FF0FF33143001F0A2
:1017900017BF00004C3001F0EFBF00004FF0FF33E7
:1017A0004C3001F0E9BF0000143001F0EBBE000046
:1017B0004FF0FF31143001F0E5BE00004C3001F075
:1017C000BBBF00004FF0FF324C3001F0B5BF00004E
:1017D000D0F8942438B5136805461978042901D047
:1017E000012038BD017C0229FAD1127901205C89DF
:1017F00090400440F4D105F1140001F07DFE024652
:101800000028EDD0D5F894544FF480732868697996
:1018100000F08CF9204638BD406BFFF7D9BF0000BF
:1018200000207047704700007FB5124B012502264B
:10183000044603600023057400F1840243602946D6
:101840008360C3600C4B0290143001934FF480739B
:10185000009601F02DFE094B04F5237229460193F1
:1018600004F14C004FF480730294009601F0F4FEF2
:1018700004B070BD10410008191800084117000895
:101880000A68202383F311880B790B3342F8230075
:101890004B79133342F823008B7913B10B3342F8A1
:1018A00023000223C0F894140374002383F31188E7
:1018B0007047000038B5037F044613B190F85430E8
:1018C000ABB90125201D0221FFF732FF04F11400FE
:1018D00025776FF0010100F09DFC84F8545004F16D
:1018E0004C006FF00101BDE8384000F093BC38BDFA
:1018F00010B5012104460430FFF71AFF00232377B7
:1019000084F8543010BD000038B50446002514306A
:1019100001F0E6FD04F14C00257701F0B5FE201D35
:1019200084F854500121FFF703FF2046BDE83840FA
:10193000FFF74EBF90F8803003F06003202B19D1E1
:1019400090F88120212A0AD0222A4FF000030ED0DD
:10195000202A0FD1084A42670722826704E0064B1B
:101960004367072383670023C367012070474367EA
:101970008367F9E7002070471C240020D0F89434D6
:1019800037B51A680446117804291AD1017C022956
:1019900017D11979012312898B40134211D100F11B
:1019A0004C05284601F030FF58B101A9284601F046
:1019B00077FED4F894440246019B2179206800F018
:1019C000C7F803B030BD000001F10B03F7B550F8C4
:1019D000234005460E46F4B1202383F3118805EB1E
:1019E0008607201D08214C34FFF7A2FEFB685B69C7
:1019F0001B6813B1204601F061FE01A9204601F0E9
:101A00004FFE024648B1019B3146284600F0A0F83F
:101A1000002383F3118803B0F0BDFB685A69126894
:101A2000002AF5D01B8A013B1340F1D105F1800259
:101A3000EAE70000133138B550F82140DCB120232B
:101A400083F31188D4F894241368527903EB82034A
:101A5000DB689B695D6845B104216018FFF768FE8B
:101A6000294604F1140001F051FD2046FFF7B0FEB5
:101A7000002383F3118838BD7047000001F04CB893
:101A8000012300F1300200F1500103700023436094
:101A900042F8043B8A42D361FAD103814381704703
:101AA00038B50446202383F31188002500F10C0388
:101AB00000F13002416043F8045B9342FBD12046C1
:101AC00001F04CF80223237085F3118838BD000023
:101AD00070B500EB8103054650690E461446DA6086
:101AE00018B110220021FFF75BFAA06918B110228B
:101AF0000021FFF755FA31462846BDE8704001F055
:101B00003FB90000038900F13002002103F0010316
:101B10000381438903F00103438100F1100343F87B
:101B2000041B9342FBD101F0C3B90000F0B40125BE
:101B300000EB810447898D40E4683D43A4694581F9
:101B400023600023A2606360F0BC01F0DFB90000F5
:101B5000F0B4012500EB810407898D40E4683D4322
:101B60006469058123600023A2606360F0BC01F01A
:101B700057BA0000022300F10C0200F1300110B549
:101B8000037004460023A0F8883080F88A3080F87B
:101B90008B300381438142F8043B8A42FBD184F8B5
:101BA0007030204601F080F863681B6823B120463E
:101BB0000021BDE81040184710BD000002784368BE
:101BC00080F88C2005221B6802700BB10421184795
:101BD00070470000436890F88C201B6802700BB1BE
:101BE000052118477047000090F8703070B5044622
:101BF00013B1002380F8703004F18002204601F018
:101C00007BF963689B6863BB94F8805015F06006AD
:101C100015D194F8813005F07F0545EA032540F29F
:101C200002339D4200F00E815BD8022D00F0DC8073
:101C30003FD8002D00F08780012D00F0CF800021DB
:101C4000204601F011FC0021204601F001FC6368F0
:101C50001B6813B1062120469847062384F870308C
:101C600070BD204698470028CED094F8872094F87D
:101C7000863043EA0223A26F934238BFA36794F9E8
:101C80008030A56F002B4FF0200380F2FD80002DE7
:101C900000F0EC80092284F8702083F31188002181
:101CA000A36F626F2046FFF753FF002383F3118871
:101CB00070BDB5F5817F00F0B180B5F5407F49D0AA
:101CC000B5F5807FBBD194F88230012BB7D1B4F841
:101CD000883023F00203A4F888306667A667E667B9
:101CE000C3E740F201639D421ED8B5F5C06F3BD2F9
:101CF000B5F5A06FA3D1B4F88030B3F5A06F0ED1C5
:101D000094F88230204684F88A3001F02BF863681A
:101D10001B6813B101212046984703232370002339
:101D20006367A367E367A0E7B5F5106F32D040F6AD
:101D300002439D4252D0B5F5006F80D104F18B0370
:101D40006367012324E004F18803E56763670223E6
:101D5000A3678AE794F88230012B7FF470AFB4F860
:101D6000883043F00203B6E794F885202046616886
:101D700094F884304D6843EA022394F8831094F871
:101D80008220A84700283FF45AAF4368636703687E
:101D9000A367A4E72378042B10D1202383F31188B1
:101DA0002046FFF7AFFE86F311886368032184F8AD
:101DB0008B601B6821700BB12046984794F88230E5
:101DC000002BACD084F88B300423237063681B682D
:101DD000002BA4D0022120469847A0E7374B636729
:101DE0000223A36700239DE794F88410204611F096
:101DF000800F01F00F010ED001F070F8012806D01D
:101E000002287FF41CAF2E4BA067636767E72D4B5A
:101E1000A567636763E701F053F8EFE794F8823052
:101E2000002B7FF40CAF94F8843013F00F013FF4D3
:101E300076AF1A06204602D501F02EFB6FE701F0BF
:101E40001FFB6CE794F88230002B7FF4F8AE94F817
:101E5000843013F00F013FF462AF1B06204602D519
:101E600001F002FB5BE701F0F3FA58E7142284F873
:101E7000702083F311882B462A4629462046FFF717
:101E800055FE85F3118870BD5DB1152284F8702070
:101E900083F311880021A36F626F2046FFF746FE8F
:101EA00003E70B2284F8702083F311882B462A461F
:101EB00029462046FFF74CFEE3E700BF40410008FB
:101EC000384100083C41000838B590F870300446AD
:101ED000152B29D8DFE803F03E28282828283E289B
:101EE000280B293928282828282828283E3E90F819
:101EF000871090F88620836F42EA01229A4214D913
:101F0000C268128AB3FBF2F502FB15356DB92023C6
:101F100083F311882B462A462946FFF719FE85F3DD
:101F200011880A2384F8703038BD142384F8703087
:101F3000202383F31188002320461A461946FFF711
:101F4000F5FD002383F3118838BDC36F03B19847B3
:101F50000023E7E7002101F087FA0021204601F085
:101F600077FA63681B6813B1062120469847062359
:101F7000D8E7000090F87020152A38B5044622D81A
:101F80000123934040F6416213421DD113F48015A2
:101F90000FD19B0217D50B2380F87030202383F3D9
:101FA00011882B462A462946FFF7D2FD85F3118872
:101FB00038BDC3689B695B682BB9C36F03B1984791
:101FC000002384F8703038BD002101F04DFA002163
:101FD000204601F03DFA63681B6813B106212046D4
:101FE00098470623EDE70000024B00221B605B6070
:101FF0009A607047AC2A0020002382680374054B66
:102000001B6899689142FBD25A6803604260106075
:1020100058607047AC2A002008B5202383F311884C
:10202000037C032B05D0042B0DD02BB983F311882F
:1020300008BD436900221A604FF0FF334361FFF788
:10204000DBFF0023F2E790E80C001A60026853609F
:10205000F2E70000002382680374054B1B6899684F
:102060009142FBD85A680360426010605860704724
:10207000AC2A0020054B196908741868026853607F
:102080001A60186101230374FEF79EB9AC2A002080
:102090004B1C30B5054687B00A4C10D0236901A807
:1020A000094A00F0D3F82846FFF7E4FF049B13B178
:1020B00001A800F007F92369586907B030BDFFF7A0
:1020C000D9FFF8E7AC2A00201920000838B50C4DDC
:1020D000044641612B6981689A68914203D8BDE842
:1020E0003840FFF789BF1846FFF786FF01232C61B0
:1020F000014623742046BDE83840FEF765B900BFAD
:10210000AC2A0020044B1A681B6990689B689842AF
:1021100094BF002001207047AC2A002010B5084C65
:10212000236820691A6854602260012223611A74AE
:10213000FFF790FF01462069BDE81040FEF744B963
:10214000AC2A00208260022202740022427470478E
:102150008368A3F17C0243F80C2C026943F83C2C01
:10216000426943F8382C074A43F81C2CC268A3F193
:10217000180043F8102C022203F8082C002203F860
:10218000072C7047E103000810B5202383F3118862
:10219000FFF7DEFF00210446FFF798FF002383F3DB
:1021A0001188204610BD0000024B1B6958610F20AA
:1021B000FFF760BFAC2A0020202383F31188FFF7CC
:1021C000F3BF000008B50146202383F311880820DF
:1021D000FFF75EFF002383F3118808BD49B1064B6A
:1021E00042681B6918605A60136043600420FFF75F
:1021F0004FBF4FF0FF307047AC2A00200368984271
:1022000006D01A680260506018465961FFF7F4BEA4
:102210007047000038B504460D462068844200D15E
:1022200038BD036823605C604561FFF7E5FEF4E7B5
:10223000054B03F114025A619A614FF0FF32DA61E3
:1022400000221A62704700BFAC2A0020F8B5036173
:1022500002291A4B0646C26038BF02215C6A184B3D
:102260001A461F4652F8145F95420AD15861986188
:102270001C620560456081600819BDE8F84001F006
:10228000E5BA186AAB68241A0C1902D3E41A2D684F
:1022900004E09C4202D2204401F0E8FAAB689C4280
:1022A000F4D86B68356073601E604FF0FF336E606A
:1022B000B460A968091BA960FB61F8BD000C00406F
:1022C000AC2A002010B41A4C234653F8141F814244
:1022D00010D0416802680A60026851609A424FF06B
:1022E0000001C16003D0936881680B4493605DF87E
:1022F000044B70470A6800209A4262615360C860CC
:1023000003D15DF8044B01F0ABBA936888680344CD
:10231000206A9360074A526A121A9342E7D9991ABF
:102320005DF8044B012998BF931C184401F09EBA34
:10233000AC2A0020000C004000207047FEE700009F
:10234000704700004FF0FF3070470000022906D0B0
:10235000032906D00129064818BF00207047054808
:102360007047032A9ABF044800EBC2000020704760
:1023700010420008C44100082424002070B59AB01F
:1023800006460846144601AD294600F095F8284651
:10239000FEF7FEFDC0B2431C5B0086E81800237008
:1023A0000323023404F8013C00231946DAB2023454
:1023B000904201D81AB070BDEA5C013304F8011CE8
:1023C00004F8022CF2E7000008B5202383F31188FB
:1023D0000348FFF7D3FA002383F3118808BD00BF39
:1023E000EC2A002010B50446052916D8DFE801F0D4
:1023F00016150316161D202383F311880E4A01219A
:10240000FFF766FB20460D4A0221FFF761FB0C48EF
:10241000FFF77AFA002383F3118810BD202383F39A
:1024200011880748FFF746FAF4E7202383F3118861
:102430000348FFF75DFAEDE74441000868410008F2
:10244000EC2A002038B50C4D0C4C2A460C4904F1FE
:102450000800FFF793FF05F1CA0204F110000949D3
:10246000FFF78CFF05F5CA7204F118000649BDE8B4
:102470003840FFF783BF00BFB42F00202424002082
:10248000944100089E410008A941000870B5044627
:1024900008460D46FEF77CFDC6B22046013403789F
:1024A0000BB9184670BD32462946FEF75BFD002881
:1024B000F3D1012070BD00002DE9F84F05460C4610
:1024C000FEF766FD2C49C6B22846FFF7DFFF08B1CC
:1024D0000236F6B229492846FFF7D8FF08B1103670
:1024E000F6B2632E0DD8DFF89080DFF89090244F7D
:1024F000DFF894A0DFF894B02E7846B92670BDE8D6
:10250000F88F29462046BDE8F84F01F0BBBD252EC7
:102510002ED1072241462846FEF724FD70B9DBF88C
:1025200000300735093444F8093CDBF8043044F83E
:10253000053C9BF8083004F8013CDDE708224946D9
:102540002846FEF70FFD98B9A21C0E4B13F8011F89
:10255000023209095345C95D02F8041C197801F0DB
:102560000F01C95D02F8031CF0D118340835C3E728
:10257000267001350134BFE730420008A941000848
:1025800042420008FFE7F11F0BE8F11F3842000844
:10259000BFF34F8F044B1A695107FCD1D3F81021B8
:1025A0005207F8D1704700BF0020005208B50D4B0C
:1025B0001B78ABB9FFF7ECFF0B4BDA68D10704D5FA
:1025C0000A4A5A6002F188325A60D3F80C21D207C5
:1025D00006D5064AC3F8042102F18832C3F8042163
:1025E00008BD00BF123200200020005223016745C1
:1025F00008B5114B1B78F3B9104B1A69510703D575
:10260000DA6842F04002DA60D3F81021520705D5AB
:10261000D3F80C2142F04002C3F80C21FFF7B8FFB9
:10262000064BDA6842F00102DA60D3F80C2142F07E
:102630000102C3F80C2108BD123200200020005214
:102640000F289ABF00F5806040040020704700000A
:102650004FF4003070470000102070470F2808B575
:102660000BD8FFF7EDFF00F500330268013204D10B
:1026700004308342F9D1012008BD002008BD0000CC
:102680000F2810B504463FD8FFF782FFFFF78EFFF3
:102690001E484FF0FF33072C4361C0F814311DD89A
:1026A0000361FFF775FF230243F02403C360C3688F
:1026B00043F08003C36003695A07FCD4FFF768FF47
:1026C0002046FFF7BDFF4FF4003100F0F7F8FFF7A9
:1026D0008FFF2046BDE81040FFF7C0BFC0F81031A3
:1026E000FFF756FFA4F108031B0243F02403C0F8D0
:1026F0000C31D0F80C3143F08003C0F80C31D0F825
:1027000010315B07FBD4D9E7002010BD0020005238
:102710002DE9F84F40EA020305460E461746DB0650
:1027200056D13446DFF8C090DFF8C0A0FFF73EFF77
:102730003B1B33441F2B04D8FFF75AFF0120BDE891
:10274000F88F20222146284601F08CFC002837D043
:1027500005F17843214A22489342224B98BF98467C
:1027600003F5827392BFD346C8469B46A3F1080384
:1027700088BF1846FFF70CFF4FF0FF3304F11C0130
:10278000A5EB040ECBF80030036843F002030360AE
:10279000231FD8F8002012F0050FFAD153F8042FA8
:1027A00099424EF80320F4D1BFF34F8FFFF7F0FEAC
:1027B0004FF0FF33CBF80030036823F002030360CF
:1027C00020222146284601F04DFC20B1FFF710FFE2
:1027D0000020BDE8F88F20352034A9E7FFFF0F0067
:1027E0000C200052102000521021005214200052E0
:1027F00010B5084C237828B153B9FFF7D7FE012351
:10280000237010BD23B12070BDE81040FFF7F0BE6B
:1028100010BD00BF1232002002440439064BD2B270
:1028200010B5904200D110BD441C00B253F82000F6
:1028300041F8040FE0B2F4E7504000580F4B30B5B8
:102840001C6F240405D41C6F1C671C6F44F40044E7
:102850001C670B4C024404392368D2B243F48073E2
:102860002360084B904200D130BD441C51F8045FF6
:1028700000B243F82050E0B2F4E700BF0044025831
:10288000004802585040005807B5012201A9002015
:10289000FFF7C2FF019803B05DF804FB13B50446CF
:1028A000FFF7F2FFA04206D002A90122002041F862
:1028B000044DFFF7C3FF02B010BD00000144BFF399
:1028C0004F8F064B884204D3BFF34F8FBFF36F8FF8
:1028D0007047C3F85C022030F4E700BF00ED00E071
:1028E000034B1B685B0142BF0122024B1A70704709
:1028F000D044025813320020014B1878704700BFB3
:1029000013320020064A536823F001035360EFF3AB
:102910000983683383F30988002383F311887047A0
:1029200030EF00E010B5202383F31188104B5B6873
:1029300013F4006318D0F1EE103AEFF309844FF06E
:10294000807344F84C3C0B4BDB6844F8083CA4F122
:10295000680383F30988FFF7D5FB18B1064B44F8E9
:10296000503C10BD054BFAE783F3118810BD00BF42
:1029700000ED00E030EF00E0F1030008F403000890
:10298000F0B5BFF34F8FBFF36F8F1D4B0021C3F81E
:102990005012BFF34F8FBFF36F8F5A6942F400326A
:1029A0005A61BFF34F8FBFF36F8FC3F88410BFF32B
:1029B0004F8FD3F8802043F6E076C2F3C904C2F308
:1029C0004E32A507520102EA060E284621464EEA7B
:1029D0000007013900F14040C3F860724F1CF6D186
:1029E000203A12F1200FEED1BFF34F8F5A6942F413
:1029F00080325A61BFF34F8FBFF36F8FF0BD00BFBE
:102A000000ED00E0FEE70000084A094B09498B424F
:102A100004D3094A0021934205D3704752F8040FAA
:102A200043F8040BF3E743F8041BF4E730440008D1
:102A3000603500206035002060350020D0F89430EB
:102A4000002230B51146D0F890409D684FF0FF301D
:102A500004EB421301329542C3F80019C3F8101970
:102A6000C3F80809C3F8001BC3F8101BC3F8080B10
:102A7000EED24FF00113C4F81C3830BD00EB8103D7
:102A80002DE9F04FD3F80CE04F1C4FEA4118DEF867
:102A900014403F03D4F800C06568D0F89020654525
:102AA0000AD30120D2F8343800FA01F123EA0101F7
:102AB000C2F83418BDE8F08FACEB0503BEF8106027
:102AC000B34228BF334602EB0806D6F81869B6B2FF
:102AD000B3EB860F13D8A6683A449946A6F1040AC8
:102AE0005AF804BFB9F1040FC2F800B002D9A9F135
:102AF0000409F5E71E442B44A6606360CCE7002080
:102B0000BDE8F08F890141F02001016103699B0656
:102B1000FCD4122000F03ABF10B50A4C2046FEF754
:102B2000AFFF094BC4F89030084BC4F89430084C00
:102B30002046FEF7A5FF074BC4F89030064BC4F8BB
:102B4000943010BD14320020000008407842000884
:102B5000B032002000000440844200080378012BBA
:102B600070B505465DD1494BD0F89040984259D197
:102B7000474B0E216520D3F8D82042F00062C3F8FD
:102B8000D820D3F8002142F00062C3F80021D3F826
:102B90000021D3F8802042F00062C3F88020D3F8EF
:102BA000802022F00062C3F88020D3F88030FEF746
:102BB000E1FB384BE360384BC4F800380023D5F80C
:102BC0009060C4F8003EC02323604FF40413A36355
:102BD0003369002BFCDA01230C20336100F0D6FEB0
:102BE0003369DB07FCD4122000F0D0FE3369002BE0
:102BF000FCDA00262846A660FFF720FF6B68C4F8C1
:102C00001068DB68C4F81468C4F81C68002B3AD15B
:102C1000224BA3614FF0FF336361A36843F00103CC
:102C2000A36070BD1E4B9842C8D1194B0E214D2098
:102C3000D3F8D82042F00072C3F8D820D3F800218E
:102C400042F00072C3F80021D3F80021D3F88020AD
:102C500042F00072C3F88020D3F8802022F0007286
:102C6000C3F88020D3F88020D3F8D82022F08062E7
:102C7000C3F8D820D3F8002122F08062C3F80021E5
:102C8000D3F8003193E7074BC3E700BF14320020AD
:102C9000004402584014004003002002003C30C0B1
:102CA000B0320020083C30C0F8B5D0F8904005465E
:102CB00000214FF000662046FFF724FFD5F894105E
:102CC00000234FF001128F684FF0FF30C4F8343802
:102CD000C4F81C2804EB431201339F42C2F8006978
:102CE000C2F8006BC2F80809C2F8080BF2D20B68F0
:102CF000D5F89020C5F898306362102313611669E7
:102D000016F01006FBD1122000F040FED4F8003877
:102D100023F4FE63C4F80038A36943F4402343F06E
:102D20001003A3610923C4F81038C4F814380B4BFE
:102D3000EB604FF0C043C4F8103B094BC4F8003BB4
:102D4000C4F81069C4F80039D5F8983003F11002BE
:102D500043F48013C5F89820A362F8BD54420008DC
:102D600040800010D0F8902090F88A10D2F80038F7
:102D700023F4FE6343EA0113C2F8003870470000F1
:102D80002DE9F0410EB20D4600EB8608D8F80C1084
:102D90000F6807F00303022B53D0032B53D03F4A95
:102DA0003F4F012B18BF1746D0F890404FEA451E01
:102DB000002205F1100C04EB0E03C3F8102B8A69F6
:102DC000002A42D04A8A05F158033A435B01E25097
:102DD0000123D4F81C2803FA0CF31343C4F81C385D
:102DE000A64400234A69CEF8103905F13F03002AB2
:102DF0003BD00A8A04EB8303898B9208012988BFA0
:102E00004A43D0F89810561841EA02422946C0F8C1
:102E1000986020465A60FFF775FED8F80C301B8A80
:102E200043EA85531F4305F148035B01E750012343
:102E3000D4F81C2803FA05F51543C4F81C58BDE85E
:102E4000F081184FB0E7184FAEE704EB4613D3F804
:102E5000002B22F40042C3F8002B0123D4F81C28D5
:102E600003FA0CF322EA0303B8E704EB83030F4AE7
:102E700004EB461629465A602046FFF743FED6F873
:102E80000039012223F4004302FA05F5C6F800399F
:102E9000D4F81C3823EA0505CFE700BF00800010F6
:102EA000008004100080081000800C100004000254
:102EB000D0F894201268C0F89820FFF7BFBD00003A
:102EC0005831D0F8903049015B5813F4004004D0D9
:102ED00013F4001F14BF0120022070474831D0F8BE
:102EE000903049015B5813F4004004D013F4001FE4
:102EF00014BF01200220704700EB8101CB68196AE2
:102F00000B6813604B6853607047000000EB81034F
:102F100030B5DD68AA691368D36019B9402B84BF46
:102F2000402313606B8A1468D0F890201C4402EB95
:102F30004110013C09B2B4FBF3F46343033323F0C3
:102F4000030343EAC44343F0C043C0F8103B2B687B
:102F500003F00303012B0ED1D2F8083802EB411025
:102F600013F4807FD0F8003B14BF43F0805343F04C
:102F70000053C0F8003B02EB4112D2F8003B43F093
:102F80000443C2F8003B30BD2DE9F041D0F8906019
:102F900005460C4606EB4113D3F8087B3A07C3F805
:102FA000087B08D5D6F814381B0704D500EB81033D
:102FB000DB685B689847FA072FD5D6F81438DB072B
:102FC0002BD505EB8403D968CCB98B69488A5E6838
:102FD000B6FBF0F200FB12628AB91868DA68904218
:102FE0000DD2121A83E81400202383F3118821469E
:102FF0002846FFF78BFF84F31188BDE8F081012399
:1030000003FA04F26B8923EA02036B81CB6823B1D4
:1030100021462846BDE8F0411847BDE8F081000090
:1030200000EB81034A0170B5DD68D0F890306C691F
:103030002668E66056BB1A444FF40020C2F8100917
:103040002A6802F00302012A0AB20ED1D3F8080856
:1030500003EB421410F4807FD4F8000914BF40F051
:10306000805040F00050C4F8000903EB4212D2F83F
:10307000000940F00440C2F800090122D3F83408E6
:1030800002FA01F10143C3F8341870BD19B9402E9A
:1030900084BF4020206020681A442E8A841940F0A2
:1030A0000050013CB4FBF6F440EAC440C6E700001F
:1030B0002DE9F041D0F8906004460D4606EB41132F
:1030C000D3F80879C3F80879FB071CD5D6F810386F
:1030D000DA0718D500EB8103D3F80CE0DEF81430E2
:1030E000D3F800C0DA6894451BD2A2EB0C024FF073
:1030F00000081A60C3F80480202383F31188FFF7C7
:103100008FFF88F311883B0618D50123D6F83428A1
:10311000AB40134212D029462046BDE8F041FFF7EC
:10312000ADBC012303FA01F2038923EA0203038100
:10313000DEF80830002BE6D09847E4E7BDE8F081E0
:103140002DE9F047D0F8905004466E69AB691E40F7
:10315000F1046E6103D5BDE8F047FEF70BBD002E0C
:1031600012DAD5F8003E9A0705D0D5F8003E23F0D4
:103170000303C5F8003ED5F80438204623F00103C8
:10318000C5F80438FEF726FD330502D52046FEF7C4
:1031900015FDB7040CD5D5F8083813F0060FEB6809
:1031A00023F470530CBF43F4105343F4A053EB606B
:1031B000300704D56368DB680BB120469847F102FD
:1031C00000F1A180B2020BD5D4F8908000274FF017
:1031D0000109D4F89430F9B29B688B4280F0D28018
:1031E000F3061AD5D4F890100A6AC2F30A1702F04F
:1031F0000F0302F4F012B2F5802F00F0EB80B2F56D
:10320000402F0AD104EB830301F58051DB68186A73
:1032100000231A469F4240F0D1803003D5F8185859
:1032200035D5E90303D500212046FFF7ADFEAA03FB
:1032300003D501212046FFF7A7FE6B0303D502212A
:103240002046FFF7A1FE2F0303D503212046FFF7F9
:103250009BFEE80203D504212046FFF795FEA90254
:1032600003D505212046FFF78FFE6A0203D506210C
:103270002046FFF789FE2B0203D507212046FFF7E2
:1032800083FEEF0103D508212046FFF77DFE700382
:1032900040F1C780E90703D500212046FFF708FF6A
:1032A000AA0703D501212046FFF702FF6B0703D5CC
:1032B00002212046FFF7FCFE2F0703D503212046FD
:1032C000FFF7F6FEEE0603D504212046FFF7F0FED9
:1032D000A80603D505212046FFF7EAFE690603D5B7
:1032E00006212046FFF7E4FE2A0603D507212046E3
:1032F000FFF7DEFEEB0540F1948020460821BDE893
:10330000F047FFF7D5BED4F890904FF000084FF08B
:10331000010AD4F894305FFA88F79B68BB42FFF447
:1033200051AF09EB4713D3F8002902F44022B2F55C
:10333000802F24D1D3F80029002A20DAD3F80029DD
:1033400042F09042C3F80029D3F80029002AFBDBA1
:103350003946D4F89000FFF7D5FB22890AFA07F323
:1033600022EA0303238104EB8703DB689B6813B124
:1033700039462046984739462046FFF77FFB08F13B
:103380000108C6E708EB4112D2F8003B03F44023E2
:10339000B3F5802F10D1D2F8003B002B0CDA6289F4
:1033A00009FA01F322EA0303638104EB8103DB687A
:1033B000DB680BB12046984701370AE713F0030F8B
:1033C00000D10A68072B03F101039EBF0270120AA5
:1033D00001301FE704EB830301F58051DA6890693F
:1033E0000268D0F808C04068A2EB000E0022104628
:1033F000974208D1DB689B699A683A449A605A6898
:1034000017445F6009E712F0030F00D10868964582
:1034100002F1010282BF8CF80000000A0CF1010CDD
:10342000E6E7BDE8F087000008B50348FFF788FE2F
:10343000BDE80840FFF776BA1432002008B503480B
:10344000FFF77EFEBDE80840FFF76CBAB0320020FF
:10345000D0F8903003EB4111D1F8003B43F4001356
:10346000C1F8003B70470000D0F8903003EB4111E9
:10347000D1F8003943F40013C1F800397047000057
:10348000D0F8903003EB4111D1F8003B23F4001346
:10349000C1F8003B70470000D0F8903003EB4111B9
:1034A000D1F8003923F40013C1F800397047000047
:1034B00030B50433039C0172002104FB0325C36172
:1034C000049B00600363059B4060C1604261026130
:1034D0008561046242628162C162436330BD000063
:1034E0000022416AC260416101616FF001018262A4
:1034F000C262FEF78FBE000003694269934203D1A6
:10350000C2680AB100207047181D7047036919602E
:103510000021C2680132C260C269134482699342C9
:10352000036124BF436A0361FEF768BE38B50446F1
:103530000D46E3683BB162690020131D1268A36267
:103540001344E36238BD237A33B929462046FEF797
:1035500045FE0028EDDA38BD6FF00100FBE7000002
:10356000C368C269013BC3604369134482699342E3
:10357000436124BF436A436100238362036B03B149
:103580001847704770B52023044683F31188866A74
:103590003EB9FFF7CBFF054618B186F311882846E0
:1035A00070BDA36AE26A13F8015B9342A36202D37F
:1035B0002046FFF7D5FF002383F31188EFE70000D3
:1035C0002DE9F84F04460E4690469946202787F38A
:1035D00011880025AA46D4F828B0BBF1000F09D104
:1035E00049462046FFF7A2FF20B18BF311882846F9
:1035F000BDE8F88FA16AA8EB050BE36A5B1A9B454F
:1036000028BF9B46BBF1400F1BD9334601F1400256
:1036100051F8040B914243F8040BF9D1A36A4036E8
:1036200040354033A362A26AE36A9A4202D320463D
:10363000FFF796FF8AF311884545D8D287F31188A2
:10364000C9E730465A46FDF783FCA36A5E445D44F1
:103650005B44A362E7E7000010B5029C04330172EB
:10366000C36103FB0421002300608362C362039BE8
:1036700040600363049BC460426102618161046233
:103680004262436310BD0000026A6FF00101C26034
:10369000426A4261026100228262C262FEF7BABDE2
:1036A000436902699A4203D1C2680AB10020704797
:1036B000184650F8043B0B6070470000C3680021B7
:1036C000C2690133C3604369134482699342436111
:1036D00024BF436A4361FEF791BD000038B504463C
:1036E0000D46E3683BB1236900201A1DA262E2691E
:1036F0001344E36238BD237A33B929462046FEF7E6
:103700006DFD0028EDDA38BD6FF00100FBE7000029
:1037100003691960C268013AC260C26913448269D0
:103720009342036124BF436A036100238362036BF6
:1037300003B118477047000070B5202304460E46B9
:1037400083F31188856A35B91146FFF7C7FF10B1B9
:1037500085F3118870BDA36A1E70A36AE26A013303
:103760009342A36204D3E16920460439FFF7D0FFF6
:10377000002080F3118870BD2DE9F84F04460D46F6
:1037800091469A464FF0200888F311880026B346E8
:10379000A76A4FB951462046FFF7A0FF20B187F333
:1037A00011883046BDE8F88FA06AA9EB0603E76AE6
:1037B0003F1A9F4228BF1F46402F1BD905F14003E7
:1037C00055F8042B9D4240F8042BF9D1A36A4036EA
:1037D0004033A362A26AE36A9A4204D3E1692046B5
:1037E0000439FFF795FF8BF311884E45D9D288F342
:1037F0001188CDE729463A46FDF7AAFBA36A3D4466
:103800003E443B44A362E5E7026943699A4203D11F
:10381000C3681BB9184670470023FBE7836A002B77
:10382000F8D0043B9B1AF5D01360C368013BC3601A
:10383000C3691A4483699A42026124BF436A0361DF
:10384000002383620123E5E700F050B9034B002217
:1038500058631A610222DA60704700BF000C004012
:103860000022014BDA607047000C0040014B5863A6
:10387000704700BF000C0040FEE7000010B5194C77
:10388000FEF7B2FBFEF7D4FC802217492046FEF774
:1038900059FC012344F8180C0374144B144AD968DA
:1038A00021F4E0610904090C0A431249DA60CA688C
:1038B00042F08072CA60104A1049C2F8B01F116805
:1038C00041F0010111601022DA77202283F82220D2
:1038D000002383F3118862B60948BDE81040FEF763
:1038E00053BC00BFD42A00209042000800ED00E045
:1038F0000003FA05F0ED00E0001000E055CEACC585
:10390000984200082DE9F84F1E4C4FF00008DFF8F0
:103910007890656904F11407D9F82430266AAA68FA
:103920009E1B96421CD34FF0200AAA68236AD5F842
:103930000CB0B61A134423622B68BB425F6063610C
:10394000C5F80C8001D1FFF78BFF88F31188286937
:10395000D8478AF311886569AB689E42E5D2DBE7F8
:103960006269BA420CD0916823628E1B9660A86887
:1039700002282CBF1818981CBDE8F84FFFF776BF37
:10398000BDE8F88FAC2A0020000C0040034B5968BA
:103990005A68521A9042FBD8704700BF001000E0EE
:1039A0004B6843608B688360CB68C3600B6943617D
:1039B0004B6903628B6943620B68036070470000C8
:1039C00008B52C4B40F2FF712B48D3F888200A43EE
:1039D000C3F88820D3F8882022F4FF6222F007027F
:1039E000C3F88820D3F88820D3F8E0200A43C3F82E
:1039F000E020D3F808210A43C3F808211F4AD3F86E
:103A000008311146FFF7CCFF1D4802F11C01FFF7FA
:103A1000C7FF1C4802F13801FFF7C2FF1A4802F144
:103A20005401FFF7BDFF194802F17001FFF7B8FF1D
:103A3000174802F18C01FFF7B3FF164802F1A80105
:103A4000FFF7AEFF144802F1C401FFF7A9FF1348C6
:103A500002F1E001FFF7A4FF114802F1FC01FFF7BA
:103A60009FFF104802F58C71FFF79AFFBDE80840F0
:103A700000F016B90044025800000258B84200088D
:103A80000004025800080258000C025800100258A6
:103A90000014025800180258001C02580020025856
:103AA000002402580028025808B500F0C9FAFFF7B0
:103AB000E5FEFEF715FFBDE80840FEF7C3BC0000B9
:103AC00070470000084B1A69920710B508D500240A
:103AD0001C61202383F31188FFF714FF84F31188FE
:103AE000BDE81040FEF71EBF000C0040124B08213D
:103AF0003220D3F8E82042F00802C3F8E820D3F8D7
:103B0000102142F00802C3F810210C4AD3F81031FA
:103B1000D36B43F00803D363C722094B9A624FF07B
:103B2000FF32DA6200229A615A63DA605A60012237
:103B30005A611A60FDF71EBC004402580010005C78
:103B4000000C0040F8B5514B0024D3F880204FF012
:103B5000FF32C3F88020D3F88010C3F88040D3F838
:103B60008010D3F88410C3F88420D3F88410C3F8ED
:103B70008440D3F88410D96F41F0FF4141F4FF0134
:103B800041F4DF4141F07F01D967D96F21F0FF4156
:103B900021F4FF0121F4DF4121F07F01D967D96FC2
:103BA000D3F888106FEA41516FEA5151C3F8881079
:103BB000D3F88810C1F30A01C3F88810D3F888102D
:103BC000D3F89010C3F89020D3F89010C3F8904029
:103BD000D3F89010D3F89410C3F89420D3F894102D
:103BE000C3F89440D3F89410D3F89810C3F89820F1
:103BF000D3F89810C3F89840D3F89810D3F88C10E5
:103C0000C3F88C20D3F88C10C3F88C40D3F88C10F8
:103C1000D3F89C10C3F89C20D3F89C20C3F89C4098
:103C2000D3F89C3000F0ECF9194B07229A60194A3E
:103C3000DA60194A1A6105225A60184A536A43F435
:103C400080335362C2F88440BFF34F8FD2F8803084
:103C500043F6E076C3F3C904C3F34E33A5075B0113
:103C600003EA060E284621464EEA0007013900F114
:103C70004040C2F874724F1CF6D1203B13F1200F64
:103C8000EED1BFF34F8FBFF36F8FF8BD00440258E2
:103C900090ED00E0000004301B00080300ED00E0A0
:103CA00001225B4B5B491A605B4B19609A605B4A6F
:103CB000DA6000221A614FF440429A619A699204D4
:103CC000FCD51A6842F480721A60554B1A6F12F4D0
:103CD000407F04D04FF480321A6700221A671A68B6
:103CE00042F001021A604E4A134611684807FCD59B
:103CF000002111611A6912F03802FBD1012119600B
:103D00004FF0804159605A67464ADA62464A1A6162
:103D10001A6842F480321A60414A134611688903D6
:103D2000FCD5116841F0800111601A68D205FCD5FC
:103D30003E4A3F499A6200225A631963A1F58021E5
:103D4000DA634B3999635A643A4A1A643A4ADA6236
:103D50001A6842F0A8521A60314B1A6802F02852D1
:103D6000B2F1285FF9D1482222219A614FF488628A
:103D7000DA6140221A624FF00052DA641A652F4A63
:103D80005A652F4A9A652F4A11601A6942F0030258
:103D90001A61234B1A6902F03802182AFAD1D3F8B3
:103DA000DC2042F00052C3F8DC20D3F8042142F0BA
:103DB0000052C3F80421D3F80421D3F8DC2042F0E8
:103DC0008042C3F8DC20D3F8042142F08042C3F8DB
:103DD0000421D3F80421D3F8DC2042F00042C3F8D8
:103DE000DC20D3F8042142F00042C3F80421D3F8C8
:103DF0000421D3F8F42042F00202C3F8F420D3F8EF
:103E00001C2142F00202C3F81C21D3F81C31704778
:103E10000881005100C000F0004802580200000173
:103E2000004402580000FF01008890081210200092
:103E30006302070147040508FD0BFF010010E000C5
:103E40000001010000200052084A08B5936811687B
:103E50000B4003F00103936023B1054A13680BB1D3
:103E600050689847BDE80840FEF75CBD80000058E8
:103E7000C0250020084A08B5936811680B4003F07C
:103E80000203936023B1054A93680BB1D068984749
:103E9000BDE80840FEF746BD80000058C025002060
:103EA000084A08B5936811680B4003F00403936057
:103EB00023B1054A13690BB150699847BDE8084022
:103EC000FEF730BD80000058C0250020084A08B524
:103ED000936811680B4003F00803936023B1054A0F
:103EE00093690BB1D0699847BDE80840FEF71ABD49
:103EF00080000058C0250020084A08B59368116862
:103F00000B4003F01003936023B1054A136A0BB111
:103F1000506A9847BDE80840FEF704BD800000588D
:103F2000C0250020174B10B59C681A68144004F493
:103F300078729A60A30604D5134A936A0BB1D06ACB
:103F40009847600604D5104A136B0BB1506B984725
:103F5000210604D50C4A936B0BB1D06B9847E20550
:103F600004D5094A136C0BB1506C9847A30504D5CE
:103F7000054A936C0BB1D06C9847BDE81040FEF732
:103F8000D1BC00BF80000058C02500201A4B10B5DE
:103F90009C681A68144004F47C429A60620504D557
:103FA000164A136D0BB1506D9847230504D5134A7B
:103FB000936D0BB1D06D9847E00404D50F4A136E92
:103FC0000BB1506E9847A10404D50C4A936E0BB107
:103FD000D06E9847620404D5084A136F0BB1506F36
:103FE0009847230404D5054A936F0BB1D06F9847C7
:103FF000BDE81040FEF796BC80000058C0250020A8
:10400000062108B50846FDF7B5F906210720FDF79A
:10401000B1F906210820FDF7ADF906210920FDF7C9
:10402000A9F906210A20FDF7A5F906211720FDF7B9
:10403000A1F906212820BDE80840FDF79BB9000042
:1040400008B5FFF77FFDFDF76BF8FDF73DFBFDF7CA
:1040500015FDFDF7E7FBFFF733FDBDE80840FFF76F
:10406000F3BB000010B501390244904201D1002099
:1040700010BD10F8013B11F8014FA342F5D0181BF9
:1040800010BD0000034611F8012B03F8012B002A94
:10409000F9D17047121012131211000001105A00CA
:1040A000031059000120580003205600EC2A00207C
:1040B0004026002053544D333248373F3F3F005392
:1040C000544D3332483734332F3735330000000036
:1040D000009600000000000000000000000000004A
:1040E0000000000000000000000000009116000821
:1040F0007D160008B9160008A5160008B1160008BC
:104100009D1600088916000875160008C5160008D7
:10411000000000009D17000889170008C517000857
:10412000B1170008BD170008A91700089517000867
:10413000811700082118000800000000010000009D
:10414000000000000200000000000000C919000883
:10415000351A000840004000842F0020942F0020D2
:10416000020000000000000003000000000000004A
:10417000791A00080000000010000000A42F0020A1
:1041800000000000010000000000000014320020C8
:10419000010102004172647550696C6F7400254220
:1041A0004F415244252D424C002553455249414C24
:1041B00025000000E52300084D23000835190008FC
:1041C000C923000843000000CC4100080902430055
:1041D000020100C0320904000001020201000524AE
:1041E0000010010524010001042402020524060038
:1041F00001070582030800FF09040100020A00000C
:104200000007050102400000070581024000000090
:1042100012000000184200081201100102000040C4
:1042200009124157000201020301000004030904BE
:1042300025424F41524425004D6174656B48373427
:104240003300303132333435363738394142434424
:104250004546000000000000E91B0008C91E0008D8
:10426000751F0008400040004C3300204C330020F4
:10427000010000005C3300208000000040010000CD
:104280000800000000010000000400000800000019
:104290006D61696E00000000B042000868330020C4
:1042A000603500200100000079380008000000009F
:1042B00069646C65000000000000802A00000000B6
:1042C000AAAAAAAA00000000FFFF00000000000048
:1042D00000A00A000000000100000000AAAAAAAA8B
:1042E00000000001FFFF00000000000000000000CF
:1042F0000000004000000000AAAAAAAA0000004096
:10430000FFFF0000000000000000000000010000AE
:1043100000000000AAAAAAAA00010000FFFF0000F6
:10432000000000000000000040804200000000008B
:10433000AAAAAAAA00404100F7FF000000000070EE
:10434000070000000000000000000000AAAAAAAABE
:1043500000000000FFFF000000000000000000005F
:104360000000000000000000AAAAAAAA00000000A5
:10437000FFFF00000000000000000000000000003F
:1043800000000000AAAAAAAA00000000FFFF000087
:10439000000000000000000000000000000000001D
:1043A000AAAAAAAA00000000FFFF00000000000067
:1043B000000000000000000000000000AAAAAAAA55
:1043C00000000000FFFF00000000000000000000EF
:1043D0000000000000000000AAAAAAAA0000000035
:1043E000FFFF0000000000000000000000000000CF
:1043F000FF00000000000000B44000083F00000083
:1044000050040000BF4000083F000000009600007C
:1044100000000800040000002C420008000000001A
:10442000000000000000000000000000000000008C
:044430000000000088
:00000001FF
